:020000021000EC
:10E000004BC000009DC000009BC0000099C00000F4
:10E0100097C0000095C0000093C0000091C00000B0
:10E020008FC000008DC0000076C5000089C00000D0
:10E0300087C0000085C0000083C0000081C00000D0
:10E040007FC000007DC000007BC0000079C00000E0
:10E0500057C3000075C0000073C0000071C000000D
:10E060006FC000006DC000006BC0000069C0000000
:10E0700067C0000065C0000063C0000061C0000010
:10E080005FC000005DC000005BC0000059C0000020
:10E0900057C0000055C0000011241FBECFEFD0E2D2
:10E0A000DEBFCDBF85B7806890E00FB6F89485BF1E
:10E0B0000FBE85BF8C9A8FE19EE40197F1F700C0F7
:10E0C00000002FB1207185B790E08F770FB6F894DC
:10E0D00085BF0FBE85BF04B603FE07C08091A001B7
:10E0E0009091A10182349C4D11F0222391F084B7CC
:10E0F000877F84BF88E10FB6F89480936000109208
:10E1000060000FBE1092A1011092A001E0E0F0E0CB
:10E11000099511E0A0E0B1E0E0EFFEEE01E00BBFF9
:10E1200002C007900D92A239B107D9F721E0A2E908
:10E13000B1E001C01D92A03AB207E1F731D0D6C6D6
:10E140005FCF84E08093E9008091E80085FD0EC0F8
:10E150008091E8008B778093E8008091E80082FD51
:10E16000F3CF8EB38111F9CF80E008958091F10053
:10E17000089593E09093E9009091E80095FF03C023
:10E180008093F10008959091E8009E779093E800C5
:10E190009091E80090FDF4CF9EB39111F9CF0895CE
:10E1A000CF93DF9300D000D000D0CDB7DEB784B7D7
:10E1B000877F84BF88E10FB6F89480936000109247
:10E1C00060000FBE90E080E80FB6F8948093610085
:10E1D000909361000FBE11E015BF82E085BF80D42F
:10E1E000269A2E9A10936F0083E0809381002E98D8
:10E1F0007894F4E08F2EA3E07A2E99249394B5E0DE
:10E200006B2E13E0212E312CAA24A394B12C8091E3
:10E210000001882309F45DC28092E9008091E80042
:10E2200082FF55C28EDF982F853419F410920001B9
:10E2300007C088E8890F823010F0943521F481DF1F
:10E240008DE097DF1DC29035D9F39C34C9F3943724
:10E2500011F484E483C0913611F489E5F2CF91344E
:10E2600091F46FDF182F6DDF90E0880F991F212F39
:10E2700030E0322F2227330F822B932BAA2797FDD2
:10E28000A095BA2FD1C1903711F483E5DACF933539
:10E2900059F40AE811E0F80181918F016ADFF1E099
:10E2A00001391F07C1F7ECC1963521F481E361DF25
:10E2B00080E3C7CF933731F482E85BDF87E959DF2A
:10E2C0008EE1BFCF953601F580E090E0DC01FC01E6
:10E2D000A0935B0070925700E89507B600FCFDCF55
:10E2E000FC01A0935B0060925700E89507B600FC24
:10E2F000FDCF9F5FAF4FBF4F811520EE920721E00A
:10E30000A207B10521F79CCF9C3651F41ADF809506
:10E3100099E0E1E0F0E0082E90935700E89590CF67
:10E32000923719F489E0F50110C0963421F489E0A0
:10E33000E0E0F0E00AC09E3419F489E0F10105C084
:10E34000913539F489E0E2E0F0E080935700849160
:10E3500078CF923631F489E50CDF81E00ADF80E086
:10E3600070CF923419F0973609F0E2C09983E9DE54
:10E37000482E512C542C4424E4DE482AE2DE182F87
:10E380008BEB810F9981823010F08FE35ACF973653
:10E3900009F04AC081E180935700E8959201512C21
:10E3A0002115310509F46CC1C0909201D090930100
:10E3B000E0909401F0909501D701C6011634D1F494
:10E3C0008529ABBFFC01879129833A83D2DE29815D
:10E3D0003A81552069F0F2E0CF0ED11CE11CF11C0E
:10E3E000C0929201D0929301E0929401F092950133
:10E3F000592417C0B695A7959795879529833A8391
:10E400005FD5B7DE82E0C80ED11CE11CF11CC092C2
:10E410009201D0929301E0929401F09295013A8199
:10E42000298121503109BCCFC0909201D090930135
:10E43000E0909401F0909501163429F05E824D82AF
:10E44000412C512C3DC0F601E0925B0070925700C8
:10E45000E89507B600FCFDCFF1CF163409F038C0BF
:10E46000552099F14091920150919301609194014E
:10E470007091950149835A836B837C8362DE242DDE
:10E4800030E0382B49815A816B817C810901FA0186
:10E4900060935B0090925700E89511244E5F5F4FA8
:10E4A0006F4F7F4F4093920150939301609394017B
:10E4B000709395015924ED81FE813197FE83ED83A0
:10E4C0008D819E81892B49F626C03BDE482EF2CFF6
:10E4D00038DE682F8091920190919301A091940170
:10E4E000B0919501B695A79597958795F1D48091B0
:10E4F000920190919301A0919401B091950102969F
:10E50000A11DB11D8093920190939301A09394015A
:10E51000B0939501D0CF163409F092CEF601E09277
:10E520005B0060925700E89507B600FCFDCF88CEEF
:10E53000933499F4C0909201D0909301E0909401AB
:10E54000F0909501FEDD90E00C01F601E0925B0099
:10E5500090925700E895112473CE933619F5C09028
:10E560009201D0909301E0909401F0909501E9DD43
:10E57000B701A601416090E00C01FA0160935B00D5
:10E5800090925700E895112492E0C90ED11CE11C2D
:10E59000F11CC0929201D0929301E0929401F0920A
:10E5A00095014ECE9D3691F4809192019091930108
:10E5B000A0919401B0919501FC01A0935B00609241
:10E5C0005700E89507B600FCFDCF3ACE923581F4AE
:10E5D0008091920190919301A0919401B091950145
:10E5E000ABBFFC0107911691812FC3DD802F29CE8F
:10E5F000943419F5A6DD682F8091920190919301D2
:10E60000A0919401B0919501B695A795979587959E
:10E610005FD48091920190919301A0919401B09167
:10E6200095010296A11DB11D8093920190939301D3
:10E63000A0939401B093950103CE9436F1F4C09069
:10E640009201D0909301E0909401F0909501D70150
:10E65000C601B695A7959795879532D48ADDE2E0F5
:10E66000CE0ED11CE11CF11CC0929201D0929301FC
:10E67000E0929401F092950103C09B3109F085CEA0
:10E680007092E9009091E8008091E8008E77809385
:10E69000E80095FD11C08091E80080FD04C08EB3B4
:10E6A0008111F9CF14C08091E8008E778093E80043
:10E6B00003C08EB3882359F08091E80080FFF9CF22
:10E6C0008092E9008091E8008B778093E800DDD3A9
:10E6D0009ECD8091E00081608093E00082E49CED1B
:10E6E0009093A1018093A0012CE088E190E00FB607
:10E6F000F894A895809360000FBE20936000FFCF30
:10E700001F920F920FB60F9211248F9380E483B95A
:10E710008F910F900FBE0F901F90189542E061EC03
:10E7200082E06BD142E161E883E067D142E160E8D9
:10E7300084E063C1809198018F778132D9F580E4BC
:10E7400083B980919901813229F0823249F1803276
:10E7500089F512C080919801813A61F58091E800B5
:10E76000877F8093E80067E070E081E091E0AED0C1
:10E770008091E8008B7711C0809198018132D1F4AB
:10E780008091E800877F8093E80067E070E081E097
:10E7900091E0F7D08091E8008E778093E8000895AB
:10E7A00080919801813231F48091E800877F8093D5
:10E7B000E80037C10895292F30E02230310539F0C3
:10E7C0002330310549F02130310561F410C08EE36A
:10E7D00090E02AE331E01EC0882371F0813089F097
:10E7E0008230A1F080E090E020E030E013C082E1D0
:10E7F00090E028E731E00EC084E090E026E331E0CD
:10E8000009C088E190E02CE131E004C082E190E0B1
:10E8100028E031E0FA0131832083089507B600FC37
:10E82000FDCFF999FECF23E0FB0180935B0020939D
:10E830005700E89507B600FCFDCF81E180935700B3
:10E84000E895089507B600FCFDCFF999FECF25E0C5
:10E85000FB0180935B0020935700E89507B600FC0E
:10E86000FDCF81E180935700E895089507B600FC3D
:10E87000FDCFF999FECF21E00A01FB0180935B00F7
:10E8800020935700E8951124089521E2FC0120937C
:10E8900057008491089529E0FC012093570084914A
:10E8A0000895E1E0F0E089E08093570084910895B5
:10E8B00007B600FCFDCFF999FECF809599E0E1E025
:10E8C000F0E0082E90935700E895089520919E015E
:10E8D00030919F012617370748F06115710539F40B
:10E8E0002091E8002E772093E80001C0B901FC01D7
:10E8F00020E06115710591F18EB38823E1F1853037
:10E90000E1F18091E80083FD3AC08091E80082FF48
:10E9100006C08091E80082FF24C080E008958091C5
:10E92000E80080FFE6CF8091F2009091F30061153E
:10E93000710551F08830910538F421912093F10050
:10E94000615071090196F3CF21E0089709F020E0AA
:10E950008091E8008E778093E800CBCF2111CCCF57
:10E96000D8CF8EB3882339F0853039F08091E80014
:10E9700083FFCFCF04C082E0089583E0089581E053
:10E9800008956115710529F42091E8002B772093F3
:10E99000E8006115710521F12EB3222351F12530D4
:10E9A00051F12091E80023FD20C02091E80022FFD2
:10E9B000F3CFFC01CF012091F2003091F300232B23
:10E9C00019F38091F1008193CF01615071096115B4
:10E9D000710581F7D9CF8EB3882359F0853059F06E
:10E9E0008091E80080FFF7CF02C081E0089580E0C9
:10E9F000089582E0089583E008958F708093E90080
:10EA0000EBEEF0E0808181608083EDEEF0E010823B
:10EA10006093EC0040838091EE00881F8827881F58
:10EA200008958091980187FD05C08091E80080FFDE
:10EA30000DC010C08091E80082FD04C08EB381112A
:10EA4000F9CF08958091E8008B7707C08EB38111CC
:10EA5000ECCF08958091E8008E778093E8000895C8
:10EA60000F931F93CF93DF9349D050D0C8EDD0E0E0
:10EA700088818F77888388818068888388818F7D6B
:10EA80008883E7EDF0E080818068808319BC1EBA3E
:10EA90001092960100EE10E0F80180818B7F808358
:10EAA00088818160888342E060E080E0A6DFE1EE5B
:10EAB000F0E080818E7F8083E2EEF0E080818160F3
:10EAC0008083808188608083F80180818E7F80834D
:10EAD000888180618883DF91CF911F910F91089584
:10EAE000E8EDF0E080818F7E8083E7EDF0E08081CB
:10EAF0008160808381E080939701B2CFE8EDF0E000
:10EB000080818C7F80831092E20008951092DA0059
:10EB10001092E10008951F920F920FB60F921124E8
:10EB20000BB60F922F933F934F935F936F937F9307
:10EB30008F939F93AF93BF93EF93FF938091DA00EE
:10EB400080FF1BC08091D80080FF17C08091DA0041
:10EB50008E7F8093DA008091D90080FF0BC08CE01B
:10EB600089BD8EE089BD09B400FEFDCF81E08EBB7A
:10EB70008BD103C019BC1EBA87D18091E10080FF00
:10EB800017C08091E20080FF13C08091E2008E7F69
:10EB90008093E2008091E20080618093E2008091A6
:10EBA000D80080628093D80019BC85E08EBB6CD100
:10EBB0008091E10084FF2EC08091E20084FF2AC092
:10EBC0008CE089BD8EE089BD09B400FEFDCF809147
:10EBD000D8008F7D8093D8008091E1008F7E809354
:10EBE000E1008091E2008F7E8093E2008091E2005C
:10EBF00081608093E20080919601882311F084E087
:10EC000007C08091E30087FF02C083E001C081E07C
:10EC10008EBB3AD18091E10083FF21C08091E20058
:10EC200083FF1DC08091E100877F8093E10082E037
:10EC30008EBB109296018091E1008E7F8093E1005F
:10EC40008091E2008E7F8093E2008091E2008061FB
:10EC50008093E20042E060E080E0CFDE15D1FF91DA
:10EC6000EF91BF91AF919F918F917F916F915F9144
:10EC70004F913F912F910F900BBE0F900FBE0F90B1
:10EC80001F9018951F93CF93DF9300D0CDB7DEB7B9
:10EC9000E8E9F1E08091F100819381E0E03AF80742
:10ECA000C9F748DD8091E80083FFDAC090919801B0
:10ECB00080919901853009F465C030F4813059F1B3
:10ECC00068F0833041F1CCC0883009F49CC08930B1
:10ECD00009F4ABC0863009F0C3C075C0903881F02C
:10ECE000923809F0BDC080919C018F708093E9003B
:10ECF0009091EB0095FB992790F91092E90001C0E3
:10ED000090E08091E800877F8093E8009093F10085
:10ED10001092F10083C0292F2D7F09F0A1C09230FD
:10ED200009F09EC090919A01911126C020919C01FA
:10ED30002F7009F495C02093E9009091EB0090FFAB
:10ED40001BC0833021F48091EB00806213C080915E
:10ED5000EB0080618093EB0081E090E0022E01C027
:10ED6000880F0A94EAF78093EA001092EA008091F3
:10ED7000EB0088608093EB001092E9008091E8003E
:10ED8000877F4FC091116CC010919A011F778091BD
:10ED9000E3008078812B8093E3008091E800877FF7
:10EDA0008093E8003EDE8091E80080FFFCCF8091F8
:10EDB000E30080688093E300112311F083E001C039
:10EDC00082E08EBB4DC09058923008F049C0AE0131
:10EDD0004F5F5F4F60919C0180919A0190919B01E0
:10EDE000EADC009709F43CC02091E800277F2093DB
:10EDF000E800BC0189819A8169DD8091E8008B7708
:10EE00008093E8002DC0903859F58091E800877F05
:10EE10008093E800809196018093F1008091E80052
:10EE20008E778093E800FDDD1BC0911119C0909191
:10EE30009A019230A8F48091E800877F8093E800DF
:10EE400090939601EEDD80919601811104C080912E
:10EE5000E30087FF02C084E001C081E08EBB5EDC7E
:10EE60008091E80083FF0AC08091E800877F80934B
:10EE7000E8008091EB0080628093EB000F900F9090
:10EE8000DF91CF911F9108950895CF938EB388237A
:10EE9000A9F08091E9008F709091EC0090FF02C082
:10EEA00090E801C090E0C92FC82B1092E900809132
:10EEB000E80083FDE7DECF70C093E900CF910895AD
:10EEC000F999FECF92BD81BDF89A992780B5089532
:10EED000262FF999FECF1FBA92BD81BD20BD0FB676
:10EEE000F894FA9AF99A0FBE01960895F894FFCF14
:10EEF000010000000000000812034C00550046000D
:10EF00004100200043004400430000001803440077
:10EF1000650061006E002000430061006D00650027
:10EF20007200610000000403090409023E000201AE
:10EF300000803209040000010202010005240010D3
:10EF400001042402020524060001070582030800CB
:10EF5000FF09040100020A00000007050402100076
:10EF600005070583021000051201100102000008C8
:10EF7000EB034A200001010200014C554641434485
:02EF800043004C
:10FFA0000C940EF40C9422F40C9436F40C9445F456
:10FFB0000C944BF40C9451F40C9458F40895089557
:06FFC00008950895089564
:10FFE000DFCFE0CFE1CFE2CFE3CFE4CFE5CFE6CF85
:08FFF000E6CFE6CFE6CFE6CF35
:08FFF80000E0010000DFFBDC6A
:040000031000E00009
:00000001FF
